:040000000000D628FE
:08000800F100030EF200831267
:1000100003130408A0000A08A1000C1922280B19D8
:1000200069280C18AF280C1BB728E0308B0083160A
:10003000031345308C008D018312031345308C056A
:100040008D01C5281508A9001608AA0001309706D9
:100050000C1127082902AB002808031C280A2A02D1
:10006000AC002D30171C303084002B088007840A28
:100070002C0803182C0A8007840A0318800A171C0E
:100080004228C5282908A7002A08A800A20BC528CD
:100090000630A200A208031957280310AF0CAE0CBB
:1000A000AD0C0310B20CB10CB00CA2034A283008FE
:1000B000B5003108B6002D08B3002E08B400AD011C
:1000C000AE01AF01B001B101B2014030A2001F1575
:1000D000C5280B11A30B87286430A300B708031DA4
:1000E000B70305091039BA003B05BC043A083B04C4
:1000F000BC053D083C063C05F7043D083C06FF3ABC
:100100003C04FF3AF8043C08BD003A08BB00A40BCD
:10011000C5280C30F41A2430A400F03086051F19CD
:10012000C52849308400250A0339A5008402000847
:100130000F39A600A60726081039260785000F30BC
:1001400087050008F039870400308A002508AA20B6
:100150008600C528820701340234043408340C10A8
:10016000B808031DB803B908031DB903C5280C134B
:10017000F4117412BD301E020318C528F415B030F6
:100180001E020318C528F411741621088A002008DD
:100190008400720E8300F10E710E0900020000004F
:1001A0000000030002000000000008008301831328
:1001B000203084008001840A841FDA28A030840063
:1001C0008001840A031DE028831710308400800119
:1001D000840A841FE728903084008001840A031D6C
:1001E000ED288313003085008600870083160313F3
:1001F0008F308100113085000E309F00F030860076
:100200000C3087008312031341309F008E018F0151
:100210004030A2006430A300053097000C110C138D
:10022000831603130C150C140C17831203130B17EE
:1002300010148B168B170830DB008030C90000309B
:10024000C600C700C800051A002D07141E30B800EC
:10025000B808031D28291F150030F500A0308400C0
:100260000C301D245530840001301D243C1A3629E1
:100270008714F701F8014C21FF218A240023771EFF
:100280003B29F701F8018710F416771E4529F7017D
:10029000F8010710771E4A29B83084008B138B1B96
:1002A0004E2933088000840A34088000840A350807
:1002B0008000840A360880008B1783160313831688
:1002C000031320082602B6002108031C210A270276
:1002D000B70020083A02B0002108031C210A3B02A3
:1002E000B100F414B11F7B29B009B1090130B00786
:1002F0000318B10AF41022082802C0002308031CC6
:10030000230A2902C1003008BC003108BD0047247F
:10031000831603133608C0003708C1005F24831614
:100320000313F41C9C2922083C07AC002308031883
:10033000230A3D07AD00A4293C082202AC003D0879
:10034000031C3D0A2302AD0024082A02C000250830
:10035000031C250A2B02C1003008BC003108BD0077
:100360004724831603133608C0003708C1005F24F2
:1003700083160313F41CC52924083C07AE00250886
:100380000318250A3D07AF00CD293C082402AE0022
:100390003D08031C3D0A2502AF000310380DBD00C7
:1003A000390DBE00F4142C08BD022D08031C2D0FBE
:1003B000BE020318E229F410BD09BE090130BD07D1
:1003C0000318BE07BF010310BD0DBE0DBF0DBD0D4F
:1003D000BE0DBF0DBD0DBE0DBF0DBC012E08C00072
:1003E0002F08C1005F2483160313753084003C0876
:1003F0008000840A3D088000831203130034073014
:100400007602031C092ABB307502031C092A7414E6
:0A04100000340830F6070024003421
:10060000741A282B7418242B34238030F4180030EB
:10061000CA007B304B020030031D132BCA00803010
:10062000F4180030CB000430CC04F41D1B2B083030
:10063000DB065B08CA044A08C6004B08C7004C0822
:10064000C8004D08C90000347410233066230034FC
:10065000B230C6002A30C700F330C800AA30C90043
:10066000771E302B0710332BD701D801D101040896
:10067000DA000430D7004930741D4E3084000A304F
:10068000D1000130741DFF3084071030D800800184
:100690000310CE0DCF0D800D0318522B5108000210
:1006A000031C552B510880024E14D80B482B0330E5
:1006B0008A0000087419103EC4238000D70B412B18
:1006C000D701D801D1015A0884000034D2000408AF
:1006D000DA004630840003308A005208D2007D23BD
:1006E000D300263A03197A2B530880005208013EA2
:1006F000840A6E2B5A088400080082073A34F334C7
:100700002A34003426343A348B342234CB34263421
:10071000E3348B34AA34003426346B34F23400349E
:1007200000342634CB348334003400342634CB34C4
:100730008B348334BA342634AA340B348234833471
:100740002634AA3402342234AA3426343A348B3480
:1007500082348234263483340B34223400342634F9
:10076000F334CB34CB3400342634B9340B34AB34CB
:100770000034263400340034003400342634BA34D3
:100780008334CB34D23426341F3982077B3441344E
:10079000DA34D934E134B934BB345134FB34F9346C
:1007A000F334AB343A34CB34BA34B2347B342234FD
:1007B000DA34BA34A334B934F9342A34FB34BB34D0
:100800007608831203178F0083120313750883126F
:1008100003178D00831603178C170C1400000000BB
:10082000831203170C0883120313CE0083120317DD
:100830000E0883120313CF00080083120313D000A5
:100840007508831203178D00831603178C130C147D
:10085000831203170C08831203138000840AF50A1D
:10086000D00B202C0800831203178C0075088D0014
:10087000831603178C130C1555308D00AA308D008C
:100880008C140C118C18422C83120313080083164D
:1008900003131030F300BF01BE0103103C1C562CA3
:1008A0004008BE0741080318410FBF07BF0CBE0C2C
:1008B000BD0CBC0CF30B4D2C8312031308008316E4
:1008C000031340083E024108031C410F3F02031C72
:1008D0006D2CFF30BC00BD00872C1030F3000310DE
:1008E000BC0DBD0DBE0DBF0D03187E2C40083E0291
:1008F0004108031C410F3F02031C852C4008BE0227
:100900004108031C410FBF02BC0AF30B6F2C83127A
:1009100003130034FF30D600D51FD601F418962CEF
:10092000CE09CF090130CE070318CF0A5508CE07EC
:1009300056080318CF0ACF07F414CF1FA62CF410C3
:0E094000CE09CF090130CE070318CF0A0034CC
:100A0000003066231E30B800B808031D042D771E81
:100A1000072DF801F701DC0105308A005C0820256C
:100A200066231E30B90005308A005C08043E771A40
:100A30002025B908031D172D5C0A0339DC000F2D92
:100A4000820705340A3428344134292D2C2D2F2DCA
:100A5000D82D0030F5007E2D0630F5007E2D0C30AF
:100A6000F5005530840001301D2400305C08781EEC
:100A7000372DF701F8012D3066231E30B900771AA3
:100A8000592DB908031D3F2D3230662374171E30CF
:100A9000B900771A5E2DB908031D492D373066233A
:100AA00074131E30B900771A5E2DB908031D532D3B
:100AB000D82D0C30F50000303324D82DF7016430E8
:100AC000B9000030CF005C08CE00F414CE1F6C2DAE
:100AD000F410CE090130CE070023B9080319782D90
:100AE000771E612DF7010130741FFF30DC075E2D8A
:100AF0000C30F5005C0855073324D82D781E7E2D68
:100B0000F701F8013E3084000F30A925B1254230AD
:100B1000840074151430A925B125A325F50A3E08D3
:100B20004207C0003F0803183F0A4307C100A3253E
:100B3000F50A42083E02C0004308031C430A3F0274
:100B4000C100A325D82D40083324F50A41083324D9
:100B50000800F701F8016623771EAC2DF701F801B4
:100B600008008B138B1BB12D3308CE003408CF0047
:100B70008B17741A282B34234A08C6004B08C70069
:100B80004C08C8004D08C900771EB12DF701F801C7
:100B90008B138B1BC82D33088000840A3408800017
:100BA000840A35088000840A360880008B17080004
:100BB000193066230A30B800B808031DDC2D071071
:020BC000DF2D27
:020C00000000F2
:020E00000000F0
:1010000000000100010001000100020002000200D6
:1010100003000300030003000400040004000400B4
:101020000500050005000600060006000600070092
:101030000700070008000800080008000900090070
:1010400009000A000A000A000A000B000B000B004E
:101050000B000C000C000C000D000D000D000D002D
:101060000E000E000E000F000F000F000F0010000A
:1010700010001000110011001100110012001200E8
:1010800012001200130013001300140014001400C7
:1010900014001500150015001600160016001600A5
:1010A0001700170017001800180018001800190082
:1010B0001900190019001A001A001A001B001B0061
:1010C0001B001B001C001C001C001D001D001D003F
:1010D0001D001E001E001E001F001F001F001F001D
:1010E00020002000200020002100210021002200FB
:1010F00022002200220023002300230024002400D9
:1011000024002400250025002500260026002600B6
:101110002600270027002700270028002800280095
:1011200029002900290029002A002A002A002B0072
:101130002B002B002B002C002C002C002D002D0050
:101140002D002D002E002E002E002E002F002F002F
:101150002F0030003000300030003100310031000D
:1011600032003200320032003300330033003400EA
:1011700034003400340035003500350036003600C8
:1011800036003600370037003700370038003800A7
:10119000380039003900390039003A003A003A0085
:1011A0003B003B003B003B003C003C003C003D0062
:1011B0003D003D003D003E003E003E003F003F0040
:1011C0003F003F004000400040004000410041001F
:1011D00041004200420042004200430043004300FD
:1011E00044004400440044004500450045004600DA
:1011F00046004600460047004700470048004800B8
:101200004800480049004900490049004A004A0096
:101210004A004B004B004B004B004C004C004C0074
:101220004D004D004D004D004E004E004E004F0051
:101230004F004F004F00500050005000510051002F
:10124000510051005200520052005300530053000D
:1012500053005400540054005500550055005500EB
:1012600056005600560056005700570057005800C9
:101270005800580058005900590059005A005A00A7
:101280005A005A005B005B005B005C005C005C0085
:101290005C005D005D005D005E005E005E005E0063
:1012A0005F005F005F006000600060006000610040
:1012B000610061006200620062006200630063001E
:1012C00063006400640064006400650065006500FC
:1012D00066006600660066006700670067006800D9
:1012E0006800680068006900690069006A006A00B7
:1012F0006A006A006B006B006B006B006C006C0096
:101300006C006D006D006D006D006E006E006E0073
:101310006F006F006F006F00700070007000710050
:10132000710071007100720072007200730073002E
:10133000730073007400740074007500750075000C
:1013400075007600760076007700770077007700EA
:1013500078007800780079007900790079007A00C7
:101360007A007A007B007B007B007B007C007C00A5
:101370007C007D007D007D007D007E007E007E0083
:101380007F007F007F00800080008000800081005F
:10139000810081008200820082008200830083003D
:1013A000830084008400840084008500850085001B
:1013B00086008600860086008700870087008800F8
:1013C0008800880088008900890089008A008A00D6
:1013D0008A008A008B008B008B008C008C008C00B4
:1013E0008C008D008D008D008E008E008E008E0092
:1013F0008F008F008F00900090009000900091006F
:10140000910091009200920092009300930093004B
:101410009300940094009400950095009500950029
:101420009600960096009700970097009700980006
:101430009800980099009900990099009A009A00E4
:101440009A009B009B009B009B009C009C009C00C2
:101450009D009D009D009E009E009E009E009F009E
:101460009F009F00A000A000A000A000A100A1007C
:10147000A100A200A200A200A200A300A300A3005A
:10148000A400A400A400A500A500A500A500A60036
:10149000A600A600A700A700A700A700A800A80014
:1014A000A800A900A900A900A900AA00AA00AA00F2
:1014B000AB00AB00AB00AC00AC00AC00AC00AD00CE
:1014C000AD00AD00AE00AE00AE00AE00AF00AF00AC
:1014D000AF00B000B000B000B100B100B100B10089
:1014E000B200B200B200B300B300B300B300B40066
:1014F000B400B400B500B500B500B600B600B60043
:10150000B600B700B700B700B800B800B800B80020
:10151000B900B900B900BA00BA00BA00BB00BB00FC
:10152000BB00BB00BC00BC00BC00BD00BD00BD00DA
:10153000BD00BE00BE00BE00BF00BF00BF00C000B7
:10154000C000C000C000C100C100C100C200C20094
:10155000C200C300C300C300C300C400C400C40071
:10156000C500C500C500C500C600C600C600C7004E
:10157000C700C700C800C800C800C800C900C9002B
:10158000C900CA00CA00CA00CB00CB00CB00CB0008
:10159000CC00CC00CC00CD00CD00CD00CE00CE00E4
:1015A000CE00CE00CF00CF00CF00D000D000D000C2
:1015B000D100D100D100D100D200D200D200D3009E
:1015C000D300D300D400D400D400D400D500D5007B
:1015D000D500D600D600D600D700D700D700D70058
:1015E000D800D800D800D900D900D900DA00DA0034
:1015F000DA00DA00DB00DB00DB00DC00DC00DC0012
:10160000DD00DD00DD00DD00DE00DE00DE00DF00ED
:10161000DF00DF00E000E000E000E000E100E100CA
:10162000E100E200E200E200E300E300E300E400A6
:10163000E400E400E400E500E500E500E600E60083
:10164000E600E700E700E700E700E800E800E80060
:10165000E900E900E900EA00EA00EA00EB00EB003B
:10166000EB00EB00EC00EC00EC00ED00ED00ED0019
:10167000EE00EE00EE00EE00EF00EF00EF00F000F5
:10168000F000F000F100F100F100F200F200F200D1
:10169000F200F300F300F300F400F400F400F500AE
:1016A000F500F500F600F600F600F600F700F7008A
:1016B000F700F800F800F800F900F900F900FA0066
:1016C000FA00FA00FA00FB00FB00FB00FC00FC0043
:1016D000FC00FD00FD00FD00FE00FE00FE00FE001F
:1016E000FF00FF00FF0000010001000101010101F6
:1016F00001010201020102010301030103010301CF
:1017000004010401040105010501050106010601AA
:101710000601070107010701070108010801080187
:101720000901090109010A010A010A010B010B0162
:101730000B010C010C010C010D010D010D010D013E
:101740000E010E010E010F010F010F01100110011A
:1017500010011101110111011201120112011201F6
:1017600013011301130114011401140115011501D2
:1017700015011601160116011701170117011801AD
:101780001801180118011901190119011A011A018A
:101790001A011B011B011B011C011C011C011D0165
:1017A0001D011D011E011E011E011F011F011F0140
:1017B0001F0120012001200121012101210122011D
:1017C00022012201230123012301240124012401F8
:1017D00025012501250126012601260127012701D2
:1017E00027012701280128012801290129012901B0
:1017F0002A012A012A012B012B012B012C012C018A
:101800002C012D012D012D012E012E012E012F0164
:101810002F012F013001300130013101310131013F
:10182000320132013201320133013301330134011B
:1018300034013401350135013501360136013601F7
:1018400037013701370138013801380139013901D1
:1018500039013A013A013A013B013B013B013C01AC
:101860003C013C013D013D013D013E013E013E0187
:101870003F013F013F014001400140014101410161
:10188000410142014201420143014301430144013C
:101890004401440145014501450146014601460117
:1018A00047014701470148014801480149014901F1
:1018B00049014A014A014A014B014B014B014C01CC
:1018C0004C014C014D014D014D014E014E014E01A7
:1018D0004F014F014F015001500150015101510181
:1018E000510152015201520153015301530154015C
:1018F0005401540155015501550156015601560137
:101900005701570157015801580158015901590110
:1019100059015A015A015A015B015B015B015C01EB
:101920005C015C015D015D015D015E015E015E01C6
:101930005F015F015F01600160016101610161019F
:101940006201620162016301630163016401640178
:101950006401650165016501660166016601670153
:10196000670167016801680168016901690169012E
:101970006A016A016A016B016B016C016C016C0107
:101980006D016D016D016E016E016E016F016F01E0
:101990006F017001700170017101710171017201BB
:1019A0007201730173017301740174017401750193
:1019B000750175017601760176017701770177016E
:1019C000780178017901790179017A017A017A0146
:1019D0007B017B017B017C017C017C017D017D0120
:1019E0007D017E017E017F017F017F0180018001F9
:1019F00080018101810181018201820182018301D3
:101A000083018401840184018501850185018601AA
:101A10008601860187018701870188018801890184
:101A2000890189018A018A018A018B018B018B015D
:101A30008C018C018D018D018D018E018E018E0135
:101A40008F018F018F01900190019101910191010E
:101A500092019201920193019301940194019401E6
:101A600095019501950196019601960197019701BF
:101A70009801980198019901990199019A019A0197
:101A80009B019B019B019C019C019C019D019D016F
:101A90009D019E019E019F019F019F01A001A00148
:101AA000A001A101A101A201A201A201A301A30120
:101AB000A301A401A401A501A501A501A601A601F8
:101AC000A601A701A701A801A801A801A901A901D0
:101AD000AA01AA01AA01AB01AB01AB01AC01AC01A7
:101AE000AD01AD01AD01AE01AE01AE01AF01AF017F
:101AF000B001B001B001B101B101B201B201B20156
:101B0000B301B301B301B401B401B501B501B5012D
:101B1000B601B601B701B701B701B801B801B90103
:101B2000B901B901BA01BA01BA01BB01BB01BC01DB
:101B3000BC01BC01BD01BD01BE01BE01BE01BF01B2
:101B4000BF01C001C001C001C101C101C201C20188
:101B5000C201C301C301C401C401C401C501C5015F
:101B6000C601C601C601C701C701C801C801C80135
:101B7000C901C901CA01CA01CA01CB01CB01CC010B
:101B8000CC01CC01CD01CD01CE01CE01CE01CF01E2
:101B9000CF01D001D001D001D101D101D201D201B8
:101BA000D201D301D301D401D401D401D501D5018F
:101BB000D601D601D601D701D701D801D801D90164
:101BC000D901D901DA01DA01DB01DB01DB01DC013A
:101BD000DC01DD01DD01DE01DE01DE01DF01DF010F
:101BE000E001E001E001E101E101E201E201E301E4
:101BF000E301E301E401E401E501E501E501E601BA
:101C0000E601E701E701E801E801E801E901E9018E
:101C1000EA01EA01EB01EB01EB01EC01EC01ED0162
:101C2000ED01EE01EE01EE01EF01EF01F001F00137
:101C3000F101F101F101F201F201F301F301F4010B
:101C4000F401F401F501F501F601F601F701F701E0
:101C5000F801F801F801F901F901FA01FA01FB01B3
:101C6000FB01FC01FC01FC01FD01FD01FE01FE0187
:101C7000FF01FF0100020002000201020102020254
:101C80000202030203020402040204020502050226
:101C900006020602070207020802080209020902F8
:101CA00009020A020A020B020B020C020C020D02CC
:101CB0000D020E020E020E020F020F02100210029F
:101CC0001102110212021202130213021402140270
:101CD0001502150215021602160217021702180243
:101CE0001802190219021A021A021B021B021C0214
:101CF0001C021D021D021D021E021E021F021F02E7
:101D000020022002210221022202220223022302B7
:101D10002402240225022502260226022702270287
:101D200028022802290229022A022A022B022B0257
:101D30002C022C022D022D022E022E022F022F0227
:101D400030023002310231023202320233023302F7
:101D500034023402350235023602360237023702C7
:101D600038023802390239023A023A023B023B0297
:101D70003C023C023D023D023E023E023F023F0267
:101D80004002400241024102420243024302440235
:101D90004402450245024602460247024702480203
:101DA0004802490249024A024A024B024C024C02D2
:101DB0004D024D024E024E024F024F02500250029F
:101DC000510252025202530253025402540255026B
:101DD0005502560257025702580258025902590238
:101DE0005A025A025B025C025C025D025D025E0204
:101DF0005E025F02600260026102610262026202D0
:101E00006302640264026502650266026702670299
:101E100068026802690269026A026B026B026C0264
:101E20006C026D026E026E026F026F02700271022E
:101E300071027202720273027402740275027602F7
:101E40007602770277027802790279027A027A02C0
:101E50007B027C027C027D027E027E027F02800287
:101E6000800281028102820283028302840285024F
:101E700085028602870287028802890289028A0215
:101E80008B028B028C028D028D028E028F028F02DA
:101E9000900291029102920293029302940295029F
:101EA0009502960297029802980299029A029A0263
:101EB0009B029C029C029D029E029F029F02A00226
:101EC000A102A102A202A302A402A402A502A602E8
:101ED000A702A702A802A902AA02AA02AB02AC02A8
:101EE000AD02AD02AE02AF02B002B002B102B20268
:101EF000B302B402B402B502B602B702B802B80225
:101F0000B902BA02BB02BC02BC02BD02BE02BF02E1
:101F1000C002C102C102C202C302C402C502C6029B
:101F2000C602C702C802C902CA02CB02CC02CD0255
:101F3000CE02CE02CF02D002D102D202D302D4020C
:101F4000D502D602D702D802D902DA02DA02DB02BF
:101F5000DC02DD02DE02DF02E002E102E202E30275
:101F6000E402E502E602E702E802EA02EB02EC0222
:101F7000ED02EE02EF02F002F102F202F302F402CD
:101F8000F602F702F802F902FA02FB02FD02FE0273
:101F9000FF02000301030303040305030603080310
:101FA00009030A030C030D030E03100311031303AB
:101FB00014031503170318031A031B031D031F0340
:101FC0002003220323032503270329032A032C03C9
:101FD0002E03300332033403360338033A033C0341
:101FE0003F0341034303460349034B034E0351039D
:101FF000550358035C03600365036B03720384039A
:022000000000DE
:023000000000CE
:084000000C0000000D000C0093
:02400E00713F00
:1042000095001A0043001D00E3000500C3001C00D8
:0A42100037001F007D0006000000CB
:00000001FF
